LX51 CODE BANKING LINKER/LOCATOR V05.01.29                                     12/09/08  00:40:54
WIN32 LX51 CODE BANKING LINKER/LOCATOR V05.01.29,  INVOKED BY:
LX51 c:\test\ir_remote\ir_remocom.obj , c:\test\ir_remote\ir_remote.DTP TO(c:\test\ir_remote\ir_r&
emote.AOF) PR(c:\test\ir_remote\ir_remote.m51) XSIZE(65536) CSIZE(65536) RS(256) RSI(128) IX MAP &



MEMORY MODEL: SMALL WITHOUT ANY FLOATING POINT ARITHMETIC


INPUT MODULES INCLUDED
  C:\TEST\IR_REMOTE\IR_REMOCOM.OBJ(IR_REMOCOM)
  C:\TEST\IR_REMOTE\IR_REMOTE.DTP(_WKRDTP_)
  c:\RIDE\Lib\RC51S.LIB(C3S)
  c:\RIDE\Lib\RC51S.LIB(HPD)
  c:\RIDE\Lib\RC51S.LIB(_C_IDATALEN)


LINK MAP OF MODULE: C:\TEST\IR_REMOTE\IR_REMOTE.AOF (IR_REMOTE)

    TYPE     BASE       LENGTH    RELOCATION     SEGMENT NAME
    ----     ----       ------    ----------     ------------

    * * * * * * *   DATA/IDATA    M E M O R Y   * * * * * * *
    REG      0000H      0008H     ABSOLUTE       "REG BANK 0"
    DATA     0008H      0006H     UNIT           ?DT?IR_REMOCOM
    DATA     000EH      0002H     OVERLAID UNIT  _DGROUP00_
             000EH      0001H     -------------  ?DT?main?IR_REMOCOM
             000FH      0001H     -------------  ?DT?_ir_data_tx?IR_REMOCOM
    IDATA    0010H      0001H     * * STACK * *  _STACK

    * * * * * * *   CODE          M E M O R Y   * * * * * * *
    CODE     0000H      0003H     ABSOLUTE       
    CODE     0003H      000FH     UNIT           ?PR?C51_STARTUP?
    CODE     0012H      000AH     UNIT           ?PR?IR_REMOCOM
    CODE     001CH      000EH     UNIT           ?PR?_delay?IR_REMOCOM
    CODE     002AH      0068H     UNIT           ?PR?ir_lead_code?IR_REMOCOM
    CODE     0092H      0061H     UNIT           ?PR?ir_end_code?IR_REMOCOM
    CODE     00F3H      007FH     UNIT           ?PR?_ir_byte_tx?IR_REMOCOM
    CODE     0172H      001FH     UNIT           ?PR?_ir_data_tx?IR_REMOCOM
    CODE     0191H      002AH     UNIT           ?PR?main?IR_REMOCOM

EXECUTABLE SUMMARY:
-------------------
    Total INTERNAL RAM storage requirement:  0010H (16)
    Total EXTERNAL RAM storage requirement:  0000H (0)
    Total     CODE     storage requirement:  01BBH (443)
Note:  Summary does not include dynamic stack requirements


REFERENCE MAP OF MODULE: C:\TEST\IR_REMOTE\IR_REMOTE.AOF (IR_REMOTE)

SEGMENT                           BI_GROUP            DT_GROUP             ID_GROUP             XD_GROUP
  +--> CALLED SEGMENT          START    LENGTH     START    LENGTH     START    LENGTH     START    LENGTH
--------------------------------------------------------------------------------------

?PR?main?IR_REMOCOM            ---------------     000EH    0001H      ---------------     ---------------
  +--> ?PR?_ir_data_tx?IR_REMOCOM

?PR?_ir_data_tx?IR_REMOCOM     ---------------     000FH    0001H     ---------------     ---------------
  +--> ?PR?ir_lead_code?IR_REMOCOM
  +--> ?PR?_ir_byte_tx?IR_REMOCOM
  +--> ?PR?ir_end_code?IR_REMOCOM

?PR?ir_lead_code?IR_REMOCOM    ---------------     ---------------     ---------------     ---------------
  +--> ?PR?_delay?IR_REMOCOM

?PR?_delay?IR_REMOCOM          ---------------     ---------------     ---------------     ---------------

?PR?_ir_byte_tx?IR_REMOCOM     ---------------     ---------------     ---------------     ---------------
  +--> ?PR?_delay?IR_REMOCOM

?PR?ir_end_code?IR_REMOCOM     ---------------     ---------------     ---------------     ---------------

SYMBOL TABLE FOR C:\TEST\IR_REMOTE\IR_REMOTE.AOF(IR_REMOCOM)
-------------------------------------------------------------

    VALUE              TYPE               NAME
    -----              ----               ----

	-------            MODULE             ir_remocom
	C:0000H            SYMBOL             _ICE_DUMMY_
	C:0191H            PUBLIC             main
	C:0172H            PUBLIC             _ir_data_tx
	C:00F3H            PUBLIC             _ir_byte_tx
	C:0092H            PUBLIC             ir_end_code
	C:002AH            PUBLIC             ir_lead_code
	C:001CH            PUBLIC             _delay
	D:000DH            PUBLIC             j
	D:000CH            PUBLIC             i
	D:0008H            PUBLIC             ir_tx_data
	C:0012H            PUBLIC             ir_num_data
	B:0093H            SYMBOL             SW2
	B:0095H            SYMBOL             SW1
	B:00A0H            SYMBOL             BUZZ
	B:0094H            SYMBOL             IR_LED
	B:0098H            SYMBOL             RI
	B:0099H            SYMBOL             TI
	B:009AH            SYMBOL             RB8
	B:009BH            SYMBOL             TB8
	B:009CH            SYMBOL             REN
	B:009DH            SYMBOL             SM2
	B:009EH            SYMBOL             SM1
	B:009FH            SYMBOL             SM0
	B:00B0H            SYMBOL             RXD
	B:00B1H            SYMBOL             TXD
	B:00B2H            SYMBOL             INT0
	B:00B3H            SYMBOL             INT1
	B:00B4H            SYMBOL             T0
	B:00B5H            SYMBOL             T1
	B:00B6H            SYMBOL             WR
	B:00B7H            SYMBOL             RD
	B:00B8H            SYMBOL             PX0
	B:00B9H            SYMBOL             PT0
	B:00BAH            SYMBOL             PX1
	B:00BBH            SYMBOL             PT1
	B:00BCH            SYMBOL             PS
	B:00A8H            SYMBOL             EX0
	B:00A9H            SYMBOL             ET0
	B:00AAH            SYMBOL             EX1
	B:00ABH            SYMBOL             ET1
	B:00ACH            SYMBOL             ES
	B:00AFH            SYMBOL             EA
	B:0088H            SYMBOL             IT0
	B:0089H            SYMBOL             IE0
	B:008AH            SYMBOL             IT1
	B:008BH            SYMBOL             IE1
	B:008CH            SYMBOL             TR0
	B:008DH            SYMBOL             TF0
	B:008EH            SYMBOL             TR1
	B:008FH            SYMBOL             TF1
	B:00D0H            SYMBOL             P
	B:00D2H            SYMBOL             OV
	B:00D3H            SYMBOL             RS0
	B:00D4H            SYMBOL             RS1
	B:00D5H            SYMBOL             F0
	B:00D6H            SYMBOL             AC
	B:00D7H            SYMBOL             CY
	D:0099H            SYMBOL             SBUF
	D:0098H            SYMBOL             SCON
	D:00B8H            SYMBOL             IP
	D:00A8H            SYMBOL             IE
	D:008DH            SYMBOL             TH1
	D:008CH            SYMBOL             TH0
	D:008BH            SYMBOL             TL1
	D:008AH            SYMBOL             TL0
	D:0089H            SYMBOL             TMOD
	D:0088H            SYMBOL             TCON
	D:0087H            SYMBOL             PCON
	D:0083H            SYMBOL             DPH
	D:0082H            SYMBOL             DPL
	D:0081H            SYMBOL             SP
	D:00F0H            SYMBOL             B
	D:00E0H            SYMBOL             ACC
	D:00D0H            SYMBOL             PSW
	D:00B0H            SYMBOL             P3
	D:00A0H            SYMBOL             P2
	D:0090H            SYMBOL             P1
	D:0080H            SYMBOL             P0
	-------            PROC               _delay
	C:001CH            LINE#              19
	C:001CH            LINE#              19
	C:001CH            LINE#              21
	C:0029H            LINE#              22
	C:0029H            LINE#              22
	-------            ENDPROC            _delay
	-------            PROC               ir_lead_code
	C:002AH            LINE#              25
	C:002AH            LINE#              25
	C:002AH            LINE#              28
	C:0034H            LINE#              29
	C:0036H            LINE#              30
	C:0038H            LINE#              31
	C:003AH            LINE#              32
	C:003CH            LINE#              33
	C:003EH            LINE#              34
	C:0040H            LINE#              35
	C:0042H            LINE#              36
	C:0044H            LINE#              37
	C:0046H            LINE#              38
	C:0048H            LINE#              39
	C:004AH            LINE#              40
	C:004CH            LINE#              41
	C:004EH            LINE#              42
	C:0050H            LINE#              43
	C:0052H            LINE#              44
	C:0054H            LINE#              45
	C:0056H            LINE#              46
	C:0058H            LINE#              47
	C:005AH            LINE#              48
	C:005CH            LINE#              49
	C:005EH            LINE#              50
	C:0060H            LINE#              51
	C:0062H            LINE#              52
	C:0064H            LINE#              53
	C:0066H            LINE#              54
	C:0068H            LINE#              55
	C:006AH            LINE#              56
	C:006CH            LINE#              57
	C:006EH            LINE#              58
	C:0070H            LINE#              59
	C:0072H            LINE#              60
	C:0074H            LINE#              61
	C:0076H            LINE#              62
	C:0078H            LINE#              63
	C:007AH            LINE#              64
	C:007CH            LINE#              65
	C:007EH            LINE#              66
	C:0080H            LINE#              67
	C:0082H            LINE#              68
	C:0084H            LINE#              28
	C:008AH            LINE#              71
	C:0091H            LINE#              72
	C:0091H            LINE#              72
	-------            ENDPROC            ir_lead_code
	-------            PROC               ir_end_code
	C:0092H            LINE#              75
	C:0092H            LINE#              75
	C:0092H            LINE#              78
	C:009CH            LINE#              79
	C:009EH            LINE#              80
	C:00A0H            LINE#              81
	C:00A2H            LINE#              82
	C:00A4H            LINE#              83
	C:00A6H            LINE#              84
	C:00A8H            LINE#              85
	C:00AAH            LINE#              86
	C:00ACH            LINE#              87
	C:00AEH            LINE#              88
	C:00B0H            LINE#              89
	C:00B2H            LINE#              90
	C:00B4H            LINE#              91
	C:00B6H            LINE#              92
	C:00B8H            LINE#              93
	C:00BAH            LINE#              94
	C:00BCH            LINE#              95
	C:00BEH            LINE#              96
	C:00C0H            LINE#              97
	C:00C2H            LINE#              98
	C:00C4H            LINE#              99
	C:00C6H            LINE#              100
	C:00C8H            LINE#              101
	C:00CAH            LINE#              102
	C:00CCH            LINE#              103
	C:00CEH            LINE#              104
	C:00D0H            LINE#              105
	C:00D2H            LINE#              106
	C:00D4H            LINE#              107
	C:00D6H            LINE#              108
	C:00D8H            LINE#              109
	C:00DAH            LINE#              110
	C:00DCH            LINE#              111
	C:00DEH            LINE#              112
	C:00E0H            LINE#              113
	C:00E2H            LINE#              114
	C:00E4H            LINE#              115
	C:00E6H            LINE#              116
	C:00E8H            LINE#              117
	C:00EAH            LINE#              118
	C:00ECH            LINE#              78
	C:00F2H            LINE#              120
	C:00F2H            LINE#              120
	-------            ENDPROC            ir_end_code
	-------            PROC               _ir_byte_tx
	C:00F3H            LINE#              124
	C:00F3H            LINE#              124
	C:00F5H            LINE#              128
	C:00F7H            LINE#              131
	C:0101H            LINE#              132
	C:0103H            LINE#              133
	C:0105H            LINE#              134
	C:0107H            LINE#              135
	C:0109H            LINE#              136
	C:010BH            LINE#              137
	C:010DH            LINE#              138
	C:010FH            LINE#              139
	C:0111H            LINE#              140
	C:0113H            LINE#              141
	C:0115H            LINE#              142
	C:0117H            LINE#              143
	C:0119H            LINE#              144
	C:011BH            LINE#              145
	C:011DH            LINE#              146
	C:011FH            LINE#              147
	C:0121H            LINE#              148
	C:0123H            LINE#              149
	C:0125H            LINE#              150
	C:0127H            LINE#              151
	C:0129H            LINE#              152
	C:012BH            LINE#              153
	C:012DH            LINE#              154
	C:012FH            LINE#              155
	C:0131H            LINE#              156
	C:0133H            LINE#              157
	C:0135H            LINE#              158
	C:0137H            LINE#              159
	C:0139H            LINE#              160
	C:013BH            LINE#              161
	C:013DH            LINE#              162
	C:013FH            LINE#              163
	C:0141H            LINE#              164
	C:0143H            LINE#              165
	C:0145H            LINE#              166
	C:0147H            LINE#              167
	C:0149H            LINE#              168
	C:014BH            LINE#              169
	C:014DH            LINE#              170
	C:014FH            LINE#              171
	C:0151H            LINE#              131
	C:0157H            LINE#              174
	C:015EH            LINE#              176
	C:0169H            LINE#              177
	C:016DH            LINE#              128
	C:0171H            LINE#              179
	C:0171H            LINE#              179
	-------            ENDPROC            _ir_byte_tx
	-------            PROC               _ir_data_tx
	D:000FH            SYMBOL             ir_num
	C:0172H            LINE#              182
	C:0172H            LINE#              182
	C:0174H            LINE#              184
	C:0177H            LINE#              185
	C:017CH            LINE#              186
	C:0181H            LINE#              187
	C:0186H            LINE#              188
	C:018DH            LINE#              189
	C:0190H            LINE#              190
	C:0190H            LINE#              190
	-------            ENDPROC            _ir_data_tx
	-------            PROC               main
	D:000EH            SYMBOL             ir_temp
	C:0191H            LINE#              193
	C:0191H            LINE#              193
	C:0191H            LINE#              197
	C:0193H            LINE#              198
	C:0195H            LINE#              202
	C:0197H            LINE#              203
	C:0199H            LINE#              205
	C:019CH            LINE#              207
	C:019FH            LINE#              208
	C:01A9H            LINE#              211
	C:01ACH            LINE#              213
	C:01AFH            LINE#              214
	C:01B9H            LINE#              230
	-------            ENDPROC            main
	-------            ENDMOD             ir_remocom
	N:00E8H            PUBLIC             TIM1_INIT
	N:0010H            PUBLIC             SIZEBUFPRINTF
	N:0100H            PUBLIC             XSTACKLEN
	N:0001H            PUBLIC             _LINKERSYMB_DUMMY_
	C:0003H            PUBLIC             ?C_START3
	D:00A0H            PUBLIC             HPD_ADDR
	N:007FH            PUBLIC             IDATALEN
	N:00FFH            PUBLIC             _INITP2?

LINK/LOCATE RUN COMPLETE,  NO ERROR FOUND.

